
D:\STM32\Program\1.11_Odchudzanie\um0427\FWLib\project\RIDE\STM3210E-EVAL\stm32f10x_dma.o:     file format elf32-littlearm
D:\STM32\Program\1.11_Odchudzanie\um0427\FWLib\project\RIDE\STM3210E-EVAL\stm32f10x_dma.o

Disassembly of section .text.DMA_DeInit:

00000000 <DMA_DeInit>:
DMA_DeInit():
D:\STM32\Program\1.11_Odchudzanie\um0427\FWLib\library\src/stm32f10x_dma.c:69
   0:	6803      	ldr	r3, [r0, #0]
D:\STM32\Program\1.11_Odchudzanie\um0427\FWLib\library\src/stm32f10x_dma.c:64
   2:	b082      	sub	sp, #8
D:\STM32\Program\1.11_Odchudzanie\um0427\FWLib\library\src/stm32f10x_dma.c:69
   4:	f023 0301 	bic.w	r3, r3, #1	; 0x1
   8:	6003      	str	r3, [r0, #0]
D:\STM32\Program\1.11_Odchudzanie\um0427\FWLib\library\src/stm32f10x_dma.c:72
   a:	2300      	movs	r3, #0
   c:	6003      	str	r3, [r0, #0]
D:\STM32\Program\1.11_Odchudzanie\um0427\FWLib\library\src/stm32f10x_dma.c:75
   e:	6043      	str	r3, [r0, #4]
D:\STM32\Program\1.11_Odchudzanie\um0427\FWLib\library\src/stm32f10x_dma.c:78
  10:	6083      	str	r3, [r0, #8]
D:\STM32\Program\1.11_Odchudzanie\um0427\FWLib\library\src/stm32f10x_dma.c:81
  12:	60c3      	str	r3, [r0, #12]
D:\STM32\Program\1.11_Odchudzanie\um0427\FWLib\library\src/stm32f10x_dma.c:83
  14:	4b2e      	ldr	r3, [pc, #184]	(d0 <DMA_DeInit+0xd0>)
  16:	4298      	cmp	r0, r3
D:\STM32\Program\1.11_Odchudzanie\um0427\FWLib\library\src/stm32f10x_dma.c:64
  18:	9001      	str	r0, [sp, #4]
D:\STM32\Program\1.11_Odchudzanie\um0427\FWLib\library\src/stm32f10x_dma.c:83
  1a:	d033      	beq.n	84 <DMA_DeInit+0x84>
  1c:	d811      	bhi.n	42 <DMA_DeInit+0x42>
  1e:	3b3c      	subs	r3, #60
  20:	4298      	cmp	r0, r3
  22:	d029      	beq.n	78 <DMA_DeInit+0x78>
  24:	d806      	bhi.n	34 <DMA_DeInit+0x34>
  26:	3b28      	subs	r3, #40
  28:	4298      	cmp	r0, r3
  2a:	d021      	beq.n	70 <DMA_DeInit+0x70>
  2c:	3314      	adds	r3, #20
  2e:	4298      	cmp	r0, r3
  30:	d020      	beq.n	74 <DMA_DeInit+0x74>
  32:	e04a      	b.n	ca <DMA_DeInit+0xca>
  34:	4b27      	ldr	r3, [pc, #156]	(d4 <DMA_DeInit+0xd4>)
  36:	4298      	cmp	r0, r3
  38:	d020      	beq.n	7c <DMA_DeInit+0x7c>
  3a:	3314      	adds	r3, #20
  3c:	4298      	cmp	r0, r3
  3e:	d01f      	beq.n	80 <DMA_DeInit+0x80>
  40:	e043      	b.n	ca <DMA_DeInit+0xca>
  42:	4b25      	ldr	r3, [pc, #148]	(d8 <DMA_DeInit+0xd8>)
  44:	4298      	cmp	r0, r3
  46:	d02c      	beq.n	a2 <DMA_DeInit+0xa2>
  48:	d808      	bhi.n	5c <DMA_DeInit+0x5c>
  4a:	f5a3 7367 	sub.w	r3, r3, #924	; 0x39c
  4e:	4298      	cmp	r0, r3
  50:	d01d      	beq.n	8e <DMA_DeInit+0x8e>
  52:	f503 7362 	add.w	r3, r3, #904	; 0x388
  56:	4298      	cmp	r0, r3
  58:	d01e      	beq.n	98 <DMA_DeInit+0x98>
  5a:	e036      	b.n	ca <DMA_DeInit+0xca>
  5c:	4b1f      	ldr	r3, [pc, #124]	(dc <DMA_DeInit+0xdc>)
  5e:	4298      	cmp	r0, r3
  60:	d029      	beq.n	b6 <DMA_DeInit+0xb6>
  62:	3314      	adds	r3, #20
  64:	4298      	cmp	r0, r3
  66:	d02b      	beq.n	c0 <DMA_DeInit+0xc0>
  68:	3b28      	subs	r3, #40
  6a:	4298      	cmp	r0, r3
  6c:	d01e      	beq.n	ac <DMA_DeInit+0xac>
  6e:	e02c      	b.n	ca <DMA_DeInit+0xca>
D:\STM32\Program\1.11_Odchudzanie\um0427\FWLib\library\src/stm32f10x_dma.c:87
  70:	4a1b      	ldr	r2, [pc, #108]	(e0 <DMA_DeInit+0xe0>)
  72:	e012      	b.n	9a <DMA_DeInit+0x9a>
D:\STM32\Program\1.11_Odchudzanie\um0427\FWLib\library\src/stm32f10x_dma.c:92
  74:	4a1a      	ldr	r2, [pc, #104]	(e0 <DMA_DeInit+0xe0>)
  76:	e015      	b.n	a4 <DMA_DeInit+0xa4>
D:\STM32\Program\1.11_Odchudzanie\um0427\FWLib\library\src/stm32f10x_dma.c:97
  78:	4a19      	ldr	r2, [pc, #100]	(e0 <DMA_DeInit+0xe0>)
  7a:	e018      	b.n	ae <DMA_DeInit+0xae>
D:\STM32\Program\1.11_Odchudzanie\um0427\FWLib\library\src/stm32f10x_dma.c:102
  7c:	4a18      	ldr	r2, [pc, #96]	(e0 <DMA_DeInit+0xe0>)
  7e:	e01b      	b.n	b8 <DMA_DeInit+0xb8>
D:\STM32\Program\1.11_Odchudzanie\um0427\FWLib\library\src/stm32f10x_dma.c:107
  80:	4a17      	ldr	r2, [pc, #92]	(e0 <DMA_DeInit+0xe0>)
  82:	e01e      	b.n	c2 <DMA_DeInit+0xc2>
D:\STM32\Program\1.11_Odchudzanie\um0427\FWLib\library\src/stm32f10x_dma.c:112
  84:	4a16      	ldr	r2, [pc, #88]	(e0 <DMA_DeInit+0xe0>)
  86:	6853      	ldr	r3, [r2, #4]
  88:	f443 0370 	orr.w	r3, r3, #15728640	; 0xf00000
  8c:	e01c      	b.n	c8 <DMA_DeInit+0xc8>
D:\STM32\Program\1.11_Odchudzanie\um0427\FWLib\library\src/stm32f10x_dma.c:117
  8e:	4a14      	ldr	r2, [pc, #80]	(e0 <DMA_DeInit+0xe0>)
  90:	6853      	ldr	r3, [r2, #4]
  92:	f043 6370 	orr.w	r3, r3, #251658240	; 0xf000000
  96:	e017      	b.n	c8 <DMA_DeInit+0xc8>
D:\STM32\Program\1.11_Odchudzanie\um0427\FWLib\library\src/stm32f10x_dma.c:122
  98:	4a12      	ldr	r2, [pc, #72]	(e4 <DMA_DeInit+0xe4>)
  9a:	6853      	ldr	r3, [r2, #4]
  9c:	f043 030f 	orr.w	r3, r3, #15	; 0xf
  a0:	e012      	b.n	c8 <DMA_DeInit+0xc8>
D:\STM32\Program\1.11_Odchudzanie\um0427\FWLib\library\src/stm32f10x_dma.c:127
  a2:	4a10      	ldr	r2, [pc, #64]	(e4 <DMA_DeInit+0xe4>)
  a4:	6853      	ldr	r3, [r2, #4]
  a6:	f043 03f0 	orr.w	r3, r3, #240	; 0xf0
  aa:	e00d      	b.n	c8 <DMA_DeInit+0xc8>
D:\STM32\Program\1.11_Odchudzanie\um0427\FWLib\library\src/stm32f10x_dma.c:132
  ac:	4a0d      	ldr	r2, [pc, #52]	(e4 <DMA_DeInit+0xe4>)
  ae:	6853      	ldr	r3, [r2, #4]
  b0:	f443 6370 	orr.w	r3, r3, #3840	; 0xf00
  b4:	e008      	b.n	c8 <DMA_DeInit+0xc8>
D:\STM32\Program\1.11_Odchudzanie\um0427\FWLib\library\src/stm32f10x_dma.c:137
  b6:	4a0b      	ldr	r2, [pc, #44]	(e4 <DMA_DeInit+0xe4>)
  b8:	6853      	ldr	r3, [r2, #4]
  ba:	f443 4370 	orr.w	r3, r3, #61440	; 0xf000
  be:	e003      	b.n	c8 <DMA_DeInit+0xc8>
D:\STM32\Program\1.11_Odchudzanie\um0427\FWLib\library\src/stm32f10x_dma.c:142
  c0:	4a08      	ldr	r2, [pc, #32]	(e4 <DMA_DeInit+0xe4>)
  c2:	6853      	ldr	r3, [r2, #4]
  c4:	f443 2370 	orr.w	r3, r3, #983040	; 0xf0000
  c8:	6053      	str	r3, [r2, #4]
D:\STM32\Program\1.11_Odchudzanie\um0427\FWLib\library\src/stm32f10x_dma.c:148
  ca:	b002      	add	sp, #8
  cc:	4770      	bx	lr
  ce:	46c0      	nop			(mov r8, r8)
  d0:	4002006c 	.word	0x4002006c
  d4:	40020044 	.word	0x40020044
  d8:	4002041c 	.word	0x4002041c
  dc:	40020444 	.word	0x40020444
  e0:	40020000 	.word	0x40020000
  e4:	40020400 	.word	0x40020400
Disassembly of section .text.DMA_Init:

00000000 <DMA_Init>:
DMA_Init():
D:\STM32\Program\1.11_Odchudzanie\um0427\FWLib\library\src/stm32f10x_dma.c:193
   0:	688a      	ldr	r2, [r1, #8]
   2:	6a0b      	ldr	r3, [r1, #32]
D:\STM32\Program\1.11_Odchudzanie\um0427\FWLib\library\src/stm32f10x_dma.c:164
   4:	b510      	push	{r4, lr}
D:\STM32\Program\1.11_Odchudzanie\um0427\FWLib\library\src/stm32f10x_dma.c:193
   6:	4313      	orrs	r3, r2
   8:	690a      	ldr	r2, [r1, #16]
D:\STM32\Program\1.11_Odchudzanie\um0427\FWLib\library\src/stm32f10x_dma.c:181
   a:	6804      	ldr	r4, [r0, #0]
D:\STM32\Program\1.11_Odchudzanie\um0427\FWLib\library\src/stm32f10x_dma.c:193
   c:	4313      	orrs	r3, r2
   e:	694a      	ldr	r2, [r1, #20]
D:\STM32\Program\1.11_Odchudzanie\um0427\FWLib\library\src/stm32f10x_dma.c:183
  10:	f424 44fe 	bic.w	r4, r4, #32512	; 0x7f00
D:\STM32\Program\1.11_Odchudzanie\um0427\FWLib\library\src/stm32f10x_dma.c:193
  14:	4313      	orrs	r3, r2
  16:	698a      	ldr	r2, [r1, #24]
D:\STM32\Program\1.11_Odchudzanie\um0427\FWLib\library\src/stm32f10x_dma.c:183
  18:	f024 04f0 	bic.w	r4, r4, #240	; 0xf0
D:\STM32\Program\1.11_Odchudzanie\um0427\FWLib\library\src/stm32f10x_dma.c:193
  1c:	4313      	orrs	r3, r2
  1e:	69ca      	ldr	r2, [r1, #28]
  20:	4313      	orrs	r3, r2
  22:	6a4a      	ldr	r2, [r1, #36]
  24:	4313      	orrs	r3, r2
  26:	6a8a      	ldr	r2, [r1, #40]
  28:	4313      	orrs	r3, r2
  2a:	4323      	orrs	r3, r4
D:\STM32\Program\1.11_Odchudzanie\um0427\FWLib\library\src/stm32f10x_dma.c:198
  2c:	6003      	str	r3, [r0, #0]
D:\STM32\Program\1.11_Odchudzanie\um0427\FWLib\library\src/stm32f10x_dma.c:202
  2e:	68cb      	ldr	r3, [r1, #12]
  30:	6043      	str	r3, [r0, #4]
D:\STM32\Program\1.11_Odchudzanie\um0427\FWLib\library\src/stm32f10x_dma.c:206
  32:	680b      	ldr	r3, [r1, #0]
  34:	6083      	str	r3, [r0, #8]
D:\STM32\Program\1.11_Odchudzanie\um0427\FWLib\library\src/stm32f10x_dma.c:210
  36:	684b      	ldr	r3, [r1, #4]
  38:	60c3      	str	r3, [r0, #12]
D:\STM32\Program\1.11_Odchudzanie\um0427\FWLib\library\src/stm32f10x_dma.c:211
  3a:	bd10      	pop	{r4, pc}
Disassembly of section .text.DMA_StructInit:

00000000 <DMA_StructInit>:
DMA_StructInit():
D:\STM32\Program\1.11_Odchudzanie\um0427\FWLib\library\src/stm32f10x_dma.c:225
   0:	2300      	movs	r3, #0
   2:	6003      	str	r3, [r0, #0]
D:\STM32\Program\1.11_Odchudzanie\um0427\FWLib\library\src/stm32f10x_dma.c:228
   4:	6043      	str	r3, [r0, #4]
D:\STM32\Program\1.11_Odchudzanie\um0427\FWLib\library\src/stm32f10x_dma.c:231
   6:	6083      	str	r3, [r0, #8]
D:\STM32\Program\1.11_Odchudzanie\um0427\FWLib\library\src/stm32f10x_dma.c:234
   8:	60c3      	str	r3, [r0, #12]
D:\STM32\Program\1.11_Odchudzanie\um0427\FWLib\library\src/stm32f10x_dma.c:237
   a:	6103      	str	r3, [r0, #16]
D:\STM32\Program\1.11_Odchudzanie\um0427\FWLib\library\src/stm32f10x_dma.c:240
   c:	6143      	str	r3, [r0, #20]
D:\STM32\Program\1.11_Odchudzanie\um0427\FWLib\library\src/stm32f10x_dma.c:243
   e:	6183      	str	r3, [r0, #24]
D:\STM32\Program\1.11_Odchudzanie\um0427\FWLib\library\src/stm32f10x_dma.c:246
  10:	61c3      	str	r3, [r0, #28]
D:\STM32\Program\1.11_Odchudzanie\um0427\FWLib\library\src/stm32f10x_dma.c:249
  12:	6203      	str	r3, [r0, #32]
D:\STM32\Program\1.11_Odchudzanie\um0427\FWLib\library\src/stm32f10x_dma.c:252
  14:	6243      	str	r3, [r0, #36]
D:\STM32\Program\1.11_Odchudzanie\um0427\FWLib\library\src/stm32f10x_dma.c:255
  16:	6283      	str	r3, [r0, #40]
D:\STM32\Program\1.11_Odchudzanie\um0427\FWLib\library\src/stm32f10x_dma.c:256
  18:	4770      	bx	lr
  1a:	46c0      	nop			(mov r8, r8)
Disassembly of section .text.DMA_Cmd:

00000000 <DMA_Cmd>:
DMA_Cmd():
D:\STM32\Program\1.11_Odchudzanie\um0427\FWLib\library\src/stm32f10x_dma.c:275
   0:	b119      	cbz	r1, a <DMA_Cmd+0xa>
D:\STM32\Program\1.11_Odchudzanie\um0427\FWLib\library\src/stm32f10x_dma.c:278
   2:	6803      	ldr	r3, [r0, #0]
   4:	f043 0301 	orr.w	r3, r3, #1	; 0x1
   8:	e002      	b.n	10 <DMA_Cmd+0x10>
D:\STM32\Program\1.11_Odchudzanie\um0427\FWLib\library\src/stm32f10x_dma.c:283
   a:	6803      	ldr	r3, [r0, #0]
   c:	f023 0301 	bic.w	r3, r3, #1	; 0x1
  10:	6003      	str	r3, [r0, #0]
D:\STM32\Program\1.11_Odchudzanie\um0427\FWLib\library\src/stm32f10x_dma.c:285
  12:	4770      	bx	lr
Disassembly of section .text.DMA_ITConfig:

00000000 <DMA_ITConfig>:
DMA_ITConfig():
D:\STM32\Program\1.11_Odchudzanie\um0427\FWLib\library\src/stm32f10x_dma.c:311
   0:	b11a      	cbz	r2, a <DMA_ITConfig+0xa>
D:\STM32\Program\1.11_Odchudzanie\um0427\FWLib\library\src/stm32f10x_dma.c:314
   2:	6803      	ldr	r3, [r0, #0]
   4:	ea41 0303 	orr.w	r3, r1, r3
   8:	e002      	b.n	10 <DMA_ITConfig+0x10>
D:\STM32\Program\1.11_Odchudzanie\um0427\FWLib\library\src/stm32f10x_dma.c:319
   a:	6803      	ldr	r3, [r0, #0]
   c:	ea23 0301 	bic.w	r3, r3, r1
  10:	6003      	str	r3, [r0, #0]
D:\STM32\Program\1.11_Odchudzanie\um0427\FWLib\library\src/stm32f10x_dma.c:321
  12:	4770      	bx	lr
Disassembly of section .text.DMA_GetCurrDataCounter:

00000000 <DMA_GetCurrDataCounter>:
DMA_GetCurrDataCounter():
D:\STM32\Program\1.11_Odchudzanie\um0427\FWLib\library\src/stm32f10x_dma.c:340
   0:	6840      	ldr	r0, [r0, #4]
D:\STM32\Program\1.11_Odchudzanie\um0427\FWLib\library\src/stm32f10x_dma.c:341
   2:	b280      	uxth	r0, r0
   4:	4770      	bx	lr
   6:	46c0      	nop			(mov r8, r8)
Disassembly of section .text.DMA_GetFlagStatus:

00000000 <DMA_GetFlagStatus>:
DMA_GetFlagStatus():
D:\STM32\Program\1.11_Odchudzanie\um0427\FWLib\library\src/stm32f10x_dma.c:408
   0:	f010 5f80 	tst.w	r0, #268435456	; 0x10000000
D:\STM32\Program\1.11_Odchudzanie\um0427\FWLib\library\src/stm32f10x_dma.c:411
   4:	bf14      	ite	ne
   6:	4b04      	ldrne	r3, [pc, #16]	(18 <DMA_GetFlagStatus+0x18>)
D:\STM32\Program\1.11_Odchudzanie\um0427\FWLib\library\src/stm32f10x_dma.c:416
   8:	4b04      	ldreq	r3, [pc, #16]	(1c <DMA_GetFlagStatus+0x1c>)
   a:	681b      	ldr	r3, [r3, #0]
   c:	4203      	tst	r3, r0
D:\STM32\Program\1.11_Odchudzanie\um0427\FWLib\library\src/stm32f10x_dma.c:433
   e:	bf0c      	ite	eq
  10:	2000      	moveq	r0, #0
  12:	2001      	movne	r0, #1
  14:	4770      	bx	lr
  16:	46c0      	nop			(mov r8, r8)
  18:	40020400 	.word	0x40020400
  1c:	40020000 	.word	0x40020000
Disassembly of section .text.DMA_ClearFlag:

00000000 <DMA_ClearFlag>:
DMA_ClearFlag():
D:\STM32\Program\1.11_Odchudzanie\um0427\FWLib\library\src/stm32f10x_dma.c:498
   0:	f010 5f80 	tst.w	r0, #268435456	; 0x10000000
D:\STM32\Program\1.11_Odchudzanie\um0427\FWLib\library\src/stm32f10x_dma.c:501
   4:	bf14      	ite	ne
   6:	4b02      	ldrne	r3, [pc, #8]	(10 <DMA_ClearFlag+0x10>)
D:\STM32\Program\1.11_Odchudzanie\um0427\FWLib\library\src/stm32f10x_dma.c:506
   8:	4b02      	ldreq	r3, [pc, #8]	(14 <DMA_ClearFlag+0x14>)
   a:	6058      	str	r0, [r3, #4]
D:\STM32\Program\1.11_Odchudzanie\um0427\FWLib\library\src/stm32f10x_dma.c:508
   c:	4770      	bx	lr
   e:	46c0      	nop			(mov r8, r8)
  10:	40020400 	.word	0x40020400
  14:	40020000 	.word	0x40020000
Disassembly of section .text.DMA_GetITStatus:

00000000 <DMA_GetITStatus>:
DMA_GetITStatus():
D:\STM32\Program\1.11_Odchudzanie\um0427\FWLib\library\src/stm32f10x_dma.c:576
   0:	f010 5f80 	tst.w	r0, #268435456	; 0x10000000
D:\STM32\Program\1.11_Odchudzanie\um0427\FWLib\library\src/stm32f10x_dma.c:579
   4:	bf14      	ite	ne
   6:	4b04      	ldrne	r3, [pc, #16]	(18 <DMA_GetITStatus+0x18>)
D:\STM32\Program\1.11_Odchudzanie\um0427\FWLib\library\src/stm32f10x_dma.c:584
   8:	4b04      	ldreq	r3, [pc, #16]	(1c <DMA_GetITStatus+0x1c>)
   a:	681b      	ldr	r3, [r3, #0]
   c:	4203      	tst	r3, r0
D:\STM32\Program\1.11_Odchudzanie\um0427\FWLib\library\src/stm32f10x_dma.c:600
   e:	bf0c      	ite	eq
  10:	2000      	moveq	r0, #0
  12:	2001      	movne	r0, #1
  14:	4770      	bx	lr
  16:	46c0      	nop			(mov r8, r8)
  18:	40020400 	.word	0x40020400
  1c:	40020000 	.word	0x40020000
Disassembly of section .text.DMA_ClearITPendingBit:

00000000 <DMA_ClearITPendingBit>:
DMA_ClearITPendingBit():
D:\STM32\Program\1.11_Odchudzanie\um0427\FWLib\library\src/stm32f10x_dma.c:665
   0:	f010 5f80 	tst.w	r0, #268435456	; 0x10000000
D:\STM32\Program\1.11_Odchudzanie\um0427\FWLib\library\src/stm32f10x_dma.c:668
   4:	bf14      	ite	ne
   6:	4b02      	ldrne	r3, [pc, #8]	(10 <DMA_ClearITPendingBit+0x10>)
D:\STM32\Program\1.11_Odchudzanie\um0427\FWLib\library\src/stm32f10x_dma.c:673
   8:	4b02      	ldreq	r3, [pc, #8]	(14 <DMA_ClearITPendingBit+0x14>)
   a:	6058      	str	r0, [r3, #4]
D:\STM32\Program\1.11_Odchudzanie\um0427\FWLib\library\src/stm32f10x_dma.c:675
   c:	4770      	bx	lr
   e:	46c0      	nop			(mov r8, r8)
  10:	40020400 	.word	0x40020400
  14:	40020000 	.word	0x40020000
